:101800006BC207B0030C0300DC0C750E080D000062
:10181000000031C361C260C25FC25EC25DC25CC211
:101820005BC2CEC059C200010100000007936000F6
:1018300000040002400000200000F89416BE19BE0B
:1018400081E08BBF1BBEDCC308951F93CF93DF9352
:10185000EC0110E0BC98C49AF89481E08BBF82E060
:101860008BBF1CD3BC9AE7EAF0E0ACEEB1E084E1B8
:10187000182E35D39091BA009F3F21F08091B90086
:1018800088231CF48BE08093B9009F3F21F0809166
:10189000B8008F3F19F485E08093B8002091B9001B
:1018A00086E3EBEBF0E0982F11929A95E9F780939D
:1018B000BB0031E03093BC003093BD001092BF00FC
:1018C0001092BE0087E69EE09093C1008093C00016
:1018D00084B38F7C84BB85B38F7C85BB80E280B969
:1018E00086B7846086BF86B7806886BF86B7832B3D
:1018F00086BF86B7806486BF032E01C0220F0A947C
:10190000EAF722B985E4E1E6F0E011928A95E9F779
:101910008FEF9FEFAFEFBFEF809361009093620076
:10192000A0936300B09364001092A600E0E0F0E0A2
:1019300084918F3F11F0219711F43093A600789491
:101940002091B80030E044E686B3992754E096959C
:1019500087955A95E1F7982F909591708091A60000
:10196000892B8093A6008091A600882311F422235E
:10197000F1F050E18091A60081114AEF1F5F14172A
:1019800050F010E088B3852788BB3F5F3A3018F0ED
:10199000312F2111215090916000809160008917B2
:1019A000E1F38091A600882329F7222319F745DF68
:1019B000DF91CF911F91089581E090E046DF089577
:1019C0001F920F920FB60F9211242F933F934F93B4
:1019D0005F936F937F938F939F93AF93BF93EF9397
:1019E000FF938BEB90E081D186B7806886BFFF9133
:1019F000EF91BF91AF919F918F917F916F915F9187
:101A00004F913F912F910F900FBE0F901F901895FF
:101A10002F923F924F925F926F927F928F929F92FE
:101A2000AF92BF92CF92DF92EF92FF920F931F93EC
:101A3000CF93DF93CDB7DEB727970FB6F894DEBF0D
:101A40000FBECDBF5C018B01FB018281803BC9F4DD
:101A500083E19CE0AA27BB27880F991FAA1F44E1B6
:101A600050E0BC01C801039620D28091B900F80172
:101A7000838384E1828381E08093A60085E190E006
:101A80000DC1813B79F59B012C5F3F4FFB016480C9
:101A9000F90171809381907C84818D3108F08CE113
:101AA000F80182833396992331F49927AC01B3016D
:101AB000CF01FBD112C0903841F49927D30101978F
:101AC0001CF005D20192FBCF08C0903409F0CDC0C4
:101AD0009927AC01B301CF01F1D1F8018281992797
:101AE0000196DCC0823B09F0C3C0DB018C918823E6
:101AF00009F0D2C01496FB01C480FD01D180E280C0
:101B0000F82E8381807CFB01138114501D3108F075
:101B10001CE1882309F093C01496BA83A983F0ECE2
:101B20002F2EFFEF3F2EFFEF4F2EFFEF5F2E2C20CB
:101B30003D204E205F20D5012D913D914D915C912E
:101B4000221633064406550619F4112309F061C024
:101B5000F5018481882309F44FC02C833D834E8393
:101B60005F83B5016B5F7F4FE0E46E2E712C812C9B
:101B7000912C620E731E841E951EFFB7FB83F89492
:101B8000E199FECF83E0F90180935700E89507B60D
:101B900000FCFDCF2615370548055905E8F401E09E
:101BA000DB018D919D91BD01AC81BD810C01FD01D9
:101BB00000935700E89511248C819D81AE81BF81EF
:101BC0000296A11DB11D8C839D83AE83BF838615B4
:101BD0009705A805B90520F385E0F9018093570022
:101BE000E89507B600FCFDCF81E180935700E895AA
:101BF0009B819FBFF5011482D5012D923D924D929C
:101C00005C92139740E450E06D917C91C50105967C
:101C10004CD1112351F1F501808191819601281B4E
:101C2000390B2A0D3B1D812F9927AC0169817A81DF
:101C3000C901059643D181E0F501848316C080383F
:101C400059F4FD013496D601812F992701971CF094
:101C500001904AD1FBCF09C0803439F4812F9927F4
:101C60001496AC01BD01C60129D180E090E016C0F8
:101C7000833B31F4DB018C91882371F4DEDD0CC0F1
:101C8000843B51F4FB018081882331F4F89488E18E
:101C900081BD88E081BDFFCF8FEF9FEF27960FB604
:101CA000F894DEBF0FBECDBFDF91CF911F910F9192
:101CB000FF90EF90DF90CF90BF90AF909F908F906C
:101CC0007F906F905F904F903F902F900895BC0150
:101CD00081E690E09DDE089511241FBECFE5D4E09B
:101CE000DEBFCDBF80E090E0B0CD0F931F93CF93C8
:101CF000DF93EC0181B1887F06B7882309F4A1C086
:101D0000803631F0883621F0803711F08837E9F4D9
:101D1000803711F0883711F41F8203C082B18E7FA3
:101D20008F8384E090E09C838B83629684E2FE0143
:101D300011928A95E9F76297CE0144969B878A872C
:101D40001C861D866F818C8517C0803811F0803904
:101D5000B1F463B18C85823230F4EA85FB85E80FFB
:101D6000F11D608305C0833218F00F7B1C821B823B
:101D70008C858F5F8C8789856DD0898762C0883814
:101D800009F45AC0883909F457C0803A09F58B81A3
:101D90009C810497D1F4ED81FE81309739F08C85D8
:101DA0008B8BCE01429609958B8B01C01B8A2B89A8
:101DB000222331F0CE0144969F878E87288B05C061
:101DC0001F861E86288B1C821B821C821B8239C0A8
:101DD000803B11F0883A81F48B819C81892B21F41E
:101DE00083E090E09C838B83198A82B18160682FA5
:101DF000898530D0898702C0883BC1F48989988958
:101E0000981710F410E010C0891719F419850F7B8A
:101E10000BC0EE85FF85E80FF11D8F5F898B108168
:101E2000612F898517D0898713B90BC0803C11F0C9
:101E3000883C21F41C821B82006403C080E090E097
:101E400004C00F7706BF81E090E0DF91CF911F9132
:101E50000F910895682797E0292F862F880F67FF35
:101E600003C0682F622701C0682F915097FFF5CFFC
:101E7000862F992708951F920F920FB60F92112463
:101E80008F93809160008F5F8093600083E882BFB2
:101E90008F910F900FBE0F901F90189583E083BF16
:101EA00012BE81E089BF78940895FB01DC0102C075
:101EB00005900D9241505040D8F70895FB01DC0188
:101EC00002C001900D9241505040D8F70895E19919
:101ED000FECFBFBBAEBBE09A11960DB20895F7DFFF
:101EE00001921A94E1F70895E199FECFBFBBAEBB12
:101EF0000DBA11960FB6F894E29AE19A0FBE0895C2
:00000001FF
